S0220000687474703A2F2F737265636F72642E736F75726365666F7267652E6E65742F1D
S12300000C9438000C94D0190C941C1A0C945F000C945F000C945F000C945F000C945F00AA
S12300200C945F000C94D71A0C945F000C94B21E0C945F000C945F000C94331A0C94F61824
S12300400C94B21F0C945F000C94311F0C945F000C9451200C9419200C945F000C945F0055
S12300600C945F000C945F000C945F000C945F0011241FBECFEFD0E1DEBFCDBF14BEA895C7
S123008088E10FB6F89480936000109260000FBE14E0A0E0B1E0E4E0F4E402C005900D92C9
S12300A0A034B107D9F716E0A0E4B4E001C01D92AB36B107E1F70E942E120C9401220C94AC
S12300C0000020E030E0D901A857BE4F0E94E321802DF901E15AFE4F80832F5F3F4F2530DD
S12300E0310589F712BC11BC089512BC11BC089512BC11BC089512BC11BC089520E931E04C
S1230100D9010E94E321802D20553140F901EA59FE4F80832F5A3E4F81E0203F380781F7AE
S123012012BC11BC089520E430E0F901EA59FE4F8081D901A05BBE4F082E0E94F0212F5F8B
S12301403F4F203A310589F712BC11BC0895CF93DF93ACE6B7E00E94EB21F093D803E09349
S1230160D703A8EAB7E00E94E321802D8093D903A0E7B7E00E94EB21F093D005E093CF05CB
S1230180A2E7B7E00E94EB21F093C105E093C005A4E7B7E00E94EB21F093B905E093B805CB
S12301A0A6E7B7E00E94EB21F093D405E093D305C0E0D0E068E777E04AE757E0DB010E94E6
S12301C0EB219F01CE01880F991FFC01EF50FB4F31832083DA010E94E321202DFE01EF5F59
S12301E0FA4F2083DA0111960E94E321202DFE01E75FFA4F2083DB0114960E94EB2186525D
S12302009C4FDC011196FC93EE932196645F7F4F4A5F5F4FC830D10589F612BC11BCDF9164
S1230220CF910895A2E0B0E00E94E321802D90E0909341018093400120914001309141013A
S1230240A3E0B0E00E94E321802D90E0982F8827820F931F9093410180934001ADEEB3E024
S12302600E94E321802D90E090934501809344012091440130914501AEEEB3E00E94E32124
S1230280802D90E0982F8827820F931F9093450180934401809140019091410190934301A7
S12302A080934201A4E0B0E00E94E321802D90E09093470180934601209146013091470147
S12302C0A5E0B0E00E94E321802D90E0982F8827820F931F9093470180934601A6E0B0E0AE
S12302E00E94E321802D90E090932501809324012091240130912501A7E0B0E00E94E3213C
S1230300802D90E0982F8827820F931F9093250180932401A1E0B0E00E94E321802D80930B
S12303204E04A8E0B0E00E94E321802D80933701A9E5B1E00E94E321802D809350018091CA
S12303405001843039F481E080933C0183E680934F0503C082E080933C01A9E0B0E00E94B6
S1230360E321802D80933601AEE0B0E00E94E321802D80934901ABE0B0E00E94E321802D42
S123038080933D01ACE0B0E00E94E321802D80933E01AFE6B1E00E94E321802D80933F017B
S12303A0A2EFB1E00E94E321802D8093C2048091C204882319F081E08093C204ADE0B0E009
S12303C00E94E321802D26E0829FC00111249093390180933801A1E7B1E00E94E321802D94
S12303E080937305A0E7B1E00E94E321802D809371058AE08093B50581E08093B305AFE880
S1230400B1E00E94E321802D809351018091510181FF05C080915101827F8093510180910D
S1230420510185FF05C0809151018F7280935101A4EFB1E00E94E321802D90E02CE231E04E
S1230440AC01429FC001439F900D529F900D11249093350580933405A5EFB1E00E94E32193
S1230460802D80933105A6EFB1E00E94E321802D80932F05A7EFB1E00E94E321802D809335
S12304802E05A8EFB1E00E94E321802D90E090932D0580932C0520912C0530912D05A9EF34
S12304A0B1E00E94E321802D90E0982F8827820F931F90932D0580932C05ABEFB1E00E94C5
S12304C0E321802D90E090935301809352012091520130915301ACEFB1E00E94E321802D82
S12304E090E0982F8827820F931F9093530180935201ADEFB1E00E94E321802D90E09093DF
S12305005501809354012091540130915501AEEFB1E00E94E321802D90E0982F8827820F04
S1230520931F9093550180935401AFEFB1E00E94E321802D90E09093990380939803209114
S1230540980330919903A0E0B2E00E94E321802D90E0982F8827820F931F9093990380933F
S1230560980320E030E0D901A25ABE4F0E94E321802DF901EA5FFD4F8083D901AE58BE4F17
S12305800E94E321802DF901E05BFA4F8083D901A458BE4F0E94E321802D808B2F5F3F4F26
S12305A02A30310501F7A7E0B2E00E94E321802D80935A01A3E0B2E00E94E321802D80935A
S12305C05B0120E030E0F901EE56FA4F84E6808BD901A45EBD4F0E94E321802D80832F5FE3
S12305E03F4F2031310579F720E030E0D901A759BE4F0E94E321802DF901E55BFE4F80839E
S12306002F5F3F4F2430310589F720E030E0D901A25DBD4F0E94E321802DF901EC5EFB4FDA
S123062080832F5F3F4F2031310589F7ADE6B1E00E94E321802D80934801A1EFB1E00E94FA
S1230640E321802D8093C104A0EFB1E00E94E321802D80934F01A6E0B2E00E94E321802DCC
S123066080934A0120E030E0D901AA54BC4F0E94E321802DF901E05FFD4F80832F5F3F4F2E
S12306802031310589F7A7ECB3E00E94E321802D80935D01A8ECB3E00E94E321802D8093D8
S12306A05E01A4EDB3E00E94E321802D8093C804A5EDB3E00E94E321802D8093C904A6ED96
S12306C0B3E00E94E321802D8093CA04A7EDB3E00E94E321802D8093CB04A8EEB3E00E9428
S12306E0E321802D90E090935701809356012091560130915701A9EEB3E00E94E321802D52
S123070090E0982F8827820F931F9093570180935601AAEEB3E00E94E321802D8093C4046E
S123072012BC11BC08958091400190914101A2E0B0E0082E0E94F021809140019091410118
S1230740892F9927A3E0B0E0082E0E94F0218091460190914701A4E0B0E0082E0E94F02163
S12307608091460190914701892F9927A5E0B0E0082E0E94F0218091240190912501A6E03B
S1230780B0E0082E0E94F0218091240190912501892F9927A7E0B0E0082E0E94F0218091D6
S12307A03701A8E0B0E0082E0E94F02180913601A9E0B0E0082E0E94F02112BC11BC08957A
S12307C080E0A1EFB1E0082E0E94F0218AE0A0EFB1E0082E0E94F0218091C204A2EFB1E03F
S12307E0082E0E94F02184E0A9E5B1E0082E0E94F02185E0ACE0B0E0082E0E94F02182E3D1
S1230800AFE6B1E0082E0E94F02124E1A1E7B1E0022E0E94F02191E0A0E7B1E0092E0E9462
S1230820F02188ECA4EFB1E0082E0E94F021A5EFB1E0092E0E94F021A6EFB1E0022E0E941B
S1230840F0218AE5A7EFB1E0082E0E94F02188EEA8EFB1E0082E0E94F02183E0A9EFB1E0F1
S1230860082E0E94F0218091520190915301ABEFB1E0082E0E94F0218091520190915301C5
S1230880892F9927ACEFB1E0082E0E94F0218091540190915501ADEFB1E0082E0E94F021D4
S12308A08091540190915501892F9927AEEFB1E0082E0E94F0218091980390919903AFEFC1
S12308C0B1E0082E0E94F0218091980390919903892F9927A0E0B2E0082E0E94F0218CED45
S12308E0A7E0B2E0082E0E94F02186EEA3E0B2E0082E0E94F0212CE132E088ECD901082EDD
S12309000E94F0212F5F3F4F82E02C323807A9F782E2AFE8B1E0082E0E94F02181E0A6E009
S1230920B2E0082E0E94F02112BC11BC0895CF92DF92EF92FF920F931F93CF93DF93C0E054
S1230940D0E0A5E0B2E00E94E321202D30E040E050E0A3EDB3E00E94E321602D6E01CC0CDC
S1230960DD1C80E292E0C80ED91EF601E080F18070E080E090E00E94602100E010E0A80155
S123098097010E94602124E630E040E050E00E94A62179018A01CA01B90124EF31E040E0F7
S12309A050E00E94602128EC30E040E050E0E20EF31E041F151FA80197010E94A621CA019F
S12309C0B9012FEF30E040E050E00E94602125E030E040E050E00E94A62112E0220F331F75
S12309E0441F551F1A95D1F7CA01B90124E630E040E050E00E94A621F60131832083219648
S1230A00C732D10509F09DCFC0E0D0E0A9ECB3E00E94E321202D30E040E050E0A3EDB3E0B0
S1230A200E94E321602D6E01CC0CDD1C8EE692E0C80ED91EF601E080F18070E080E090E0A4
S1230A400E94602100E010E0A80197010E94602124E630E040E050E00E94A62179018A0163
S1230A60CA01B90124EF31E040E050E00E94602128EC30E040E050E0E20EF31E041F151F8A
S1230A80A80197010E94A621CA01B9012FEF30E040E050E00E94602125E030E040E050E01D
S1230AA00E94A621A2E0220F331F441F551FAA95D1F7CA01B90124E630E040E050E00E9455
S1230AC0A621F601318320832196C732D10509F09DCFC0E0D0E0AAECB3E00E94E321202DA6
S1230AE030E040E050E0A3EDB3E00E94E321602D6E01CC0CDD1C8CEB92E0C80ED91EF6014F
S1230B00E080F18070E080E090E00E94602100E010E0A80197010E94602124E630E040E04F
S1230B2050E00E94A62179018A01CA01B90124EF31E040E050E00E94602128EC30E040E0B3
S1230B4050E0E20EF31E041F151FA80197010E94A621CA01B9012FEF30E040E050E00E94BA
S1230B60602125E030E040E050E00E94A621E2E0220F331F441F551FEA95D1F7CA01B9013A
S1230B8024E630E040E050E00E94A621F601318320832196C732D10509F09DCFC0E0D0E0F5
S1230BA0A4E0B2E00E94E321202D30E040E050E0A3EDB3E00E94E321602D6E01CC0CDD1C32
S1230BC08AE093E0C80ED91EF601E080F18070E080E090E00E94602100E010E0A80197014B
S1230BE00E94602124E630E040E050E00E94A62179018A01CA01B90124EF31E040E050E0FD
S1230C000E94602128EC30E040E050E0E20EF31E041F151FA80197010E94A621CA01B901B2
S1230C202FEF30E040E050E00E94602125E030E040E050E00E94A62162E0220F331F441F19
S1230C40551F6A95D1F7CA01B90124E630E040E050E00E94A621F601318320832196C732FF
S1230C60D10509F09DCFDF91CF911F910F91FF90EF90DF90CF9008950895EAE7F0E01082CC
S1230C8010927C0080E880BF87EE808311B808950F931F93CF93DF93282F30E0F901EE0F27
S1230CA0FF1FEA5DFE4F0081118143E0033F140718F0E2E3F0E04CC053E00F3D150718F09F
S1230CC0EAE0F0E045C0C0E0D0E087E290E0A901489F9001499F300D589F300D1124D901BE
S1230CE0AC0FBD1FAA0FBB1FA05EBD4F8D919C9111978017910730F5FE013197E20FF31FAB
S1230D00EE0FFF1FE05EFD4F20813181608171814D915C91FE01EE0FFF1FEE0FFF1FEC0F09
S1230D20FD1F3596201B310BC901880F991F880F991F641B750B820F931F0E947F21E60F70
S1230D40F71F06C02196C732D10549F6E8ECF0E0CF01DF91CF911F910F9108950F931F9369
S1230D60CF93DF93AC01E0E0F0E0EF01CC0FDD1FDE01A85ABC4F8D919C91119748175907F9
S1230D80C0F56D917C913197EE0FFF1FDF01A85ABC4F8D919C911197681B790B8D919C917A
S1230DA0C059DC4F28813981E059FC4F00811181481B590B84E690E0DC014A9FC0014B9FDF
S1230DC0900D5A9F900D11240E947F21201B310B0190F081E02D629FC001639F900D729F6D
S1230DE0900D112464E670E00E947F216E0F7F1F09C03196EA30F10509F0B7CF609184038F
S1230E0070918503CB01DF91CF911F910F9108958091500490915104282F205527FF0AC025
S1230E208091380190913901BC01660F771F680F791F1EC02F312CF0609138017091390173
S1230E4017C04091380150913901332727FD309588E290E0821B930B9C01249FC001259F55
S1230E60900D349F900D11246AE070E00E947F21CB0108950F931F93CF93DF93AC01809101
S1230E809B0390919C034817590718F4E0EFF0E057C08091B7039091B8038417950718F485
S1230EA0E0E0F0E04DC0E1E0F0E0EF01CC0FDD1FDE01A556BC4F8D919C91119748175907A2
S1230EC0C0F56D917C913197EE0FFF1FDF01A556BC4F8D919C911197681B790B8D919C9140
S1230EE0E754FC4F20813181C754DC4F08811981481B590B84E690E0DC014A9FC0014B9F9A
S1230F00900D5A9F900D11240E947F21201B310B0190F081E02D629FC001639F900D729F2B
S1230F20900D112464E670E00E947F21E61BF70B07C03196EE30F10509F0B7CFEEEFF0E02E
S1230F40CF01DF91CF911F910F9108958091CF0487FF0BC08CED95E09093590180935801F4
S1230F601092DB041092DA042AC08091CF0484FF09C08CED95E0909359018093580184E611
S1230F8090E019C08091CF0483FF09C08CED95E090935901809358018AEF90E00CC0809138
S1230FA0CF0480FF0CC08CED95E0909359018093580184EF91E09093DB048093DA04F894D5
S1230FC08091BD049091BE048A5A9A4AC1F08091BD049091BE048555954589F078948091E0
S1230FE09005909191058064909391058093900584EF91E090935901809358010AC07894B9
S123100080919005909191058F7B9093910580939005F8948091BF049091C0048F5F9F4FE3
S123102089F0789480919005909191058068909391058093900584EF91E09093590180930D
S123104058010AC0789480919005909191058F7790939105809390058091580190915901B4
S1231060892B91F1429A2091DA043091DB042115310511F4429A15C08091D8049091D9041E
S1231080029778F488B18695869580958170880F880F98B19B7F982B98B93093D9042093DA
S12310A0D8048091D8049091D90401979093D9048093D8048091580190915901019790933E
S12310C0590180935801089542981092DB041092DA040895CF93DF93809190059091910500
S12310E09F77909391058093900580910505882319F4E0E0F0E025C02091B5043091B60448
S12311008091B8059091B90540E050E08217930710F441E050E0FA01452B99F08091050537
S1231120853038F4833078F4813039F0823049F406C0853031F460E807C064E005C068E0E2
S123114003C060E001C060E180910605882359F18091B5049091B6042091B8053091B905E3
S12311604091D3055091D405241B350B2817390708F4F260F1FF17C080910605833081F0B5
S1231180843028F4813041F0823069F407C0843039F0853041F406C0646005C0686003C022
S12311A0606101C06068339958C080910705882329F12091B5043091B6048091CF05909130
S12311C0D0058217930708F4E260E1FF17C080910705833081F0843028F4813041F0823069
S12311E069F407C0843039F0853041F406C0646005C0686003C0606101C0606880910805BE
S1231200882359F18091B5049091B6042091CF053091D0054091C0055091C105241B350B59
S12312202817390708F4F460F2FF17C080910805833081F0843028F4813041F0823069F410
S123124007C0843039F0853041F406C0646005C0686003C0606101C0606880919005909111
S123126091059F013327269537952227282B392B309391052093900580910105882309F4F3
S12312804BC080910905882361F42091E1043091E2048091F1049091F2048217930768F437
S12312A00BC02091E1043091E2048091F1049091F2042817390708F4E061E4FF2DC0809168
S12312C001058330D9F0843028F4813041F0823019F507C0843039F08530F1F411C0646043
S12312E01BC0686019C02091B5043091B6048091DA039091DB038217930770F460610CC078
S12313002091B5043091B6048091DA039091DB038217930708F4606880910205882309F440
S12313204BC080910A05882361F42091E3043091E4048091F3049091F4048217930768F48D
S12313400BC02091E3043091E4048091F3049091F4042817390708F4E062E5FF2DC08091BD
S123136002058330D9F0843028F4813041F0823019F507C0843039F08530F1F411C06460A1
S12313801BC0686019C02091B5043091B6048091DC039091DD038217930770F460610CC0D3
S12313A02091B5043091B6048091DC039091DD038217930708F4606880910305882309F49B
S12313C04BC080910B05882361F42091E5043091E6048091F5049091F6048217930768F4E4
S12313E00BC02091E5043091E6048091F5049091F6042817390708F4E064E6FF2DC0809112
S123140003058330D9F0843028F4813041F0823019F507C0843039F08530F1F411C06460FF
S12314201BC0686019C02091B5043091B6048091DE039091DF038217930770F460610CC02E
S12314402091B5043091B6048091DE039091DF038217930708F460681092B104F093CE040B
S1231460E093CD046093CF048091CF0487FF17C020E030E00CC0F0E08091D7039091D8038A
S12314800196EE0FFF1FEF5EFA4F91838083E22F8091D9032F5F3F4FE81768F32EC0809176
S12314A0CF0482FF2AC080914104282F30E0F901E050FF4FE081F0E0EE0FFF1FE15FFA4FE0
S12314C080819181892BC9F4C90101966CE070E00E949321FC0180934104F0E0E050FF4F8E
S12314E0E081F0E08091D7039091D8030196EE0FFF1FE15FFA4F9183808340E050E051C01D
S1231500AE2FB0E09D01220F331FF901E651FC4F0190F081E02D9081FD01EA50FC4F808119
S12315209823E901CF5EDA4F992301F588819981F901E450FC4FED01C85FDB4F892B39F042
S12315400190F081E02D80819881892B07C00190F081E02D90818881809589238083AA0F3D
S1231560BB1FAE5BBB4F1D921C9219C088819981892BA9F0F901EE5BFB4F8081918101969D
S1231580918380832091D7033091D8038217930730F01982188210924304109242044F5F02
S12315A05F4FE42F8091D903481708F4A9CFDF91CF910895809124019091250193FF6FC0FB
S12315C0339B06C08091D4048F5F8093D40402C01092D4048091D404853108F451C0209118
S12315E0B5043091B60480919803909199038217930778F48091CD049091CE0482609093D1
S1231600CE048093CD048091CF0480618093CF0409C08091CD049091CE048D7F9093CE04C6
S12316208093CD0480914E0483FF16C08091B5049091B604815D974078F08091CD04909142
S1231640CE0484609093CE048093CD048091CF0482608093CF0409C08091CD049091CE04AD
S12316608B7F9093CE048093CD048091D10490E09093D3048093D20484E38093D40408955B
S12316808091D2049091D304892B49F08091D2049091D30401979093D3048093D204089583
S12316A09C0180914E0484FF1BC022533040C901F3E0880F991FFA95E1F7220F331F280FD6
S12316C0391F2455354F442737FD4095542F60E579E784E090E00E94C821822F90E00895F8
S12316E080914E0485FD03C084E690E0089522533040C90173E0880F991F7A95E1F7220F5E
S1231700331F280F391F2455354F442737FD4095542F60E579E784E090E00E94C8212C5967
S12317202695822F90E00895A89582E50E94A62083E10E94A6208091B5049091B604892FF7
S123174099270E94A6208091B5049091B6040E94A62080915204909153040E94A6208091F8
S12317605404909155040E94A62080915004909151040E94A62080915E0490915F040E944F
S1231780A62080915C0490915D040E94A62080915804909159040E94A6208091BB049091E0
S12317A0BC0460913C0170E00E947F21CB010E94A6208091BA040E94A6208091B9040E94CA
S12317C0A62020919005309191058091490590914A05F3E096958795FA95E1F78170232F0F
S12317E03327822B0E94A62080919005909191050E94A620809130050E94A6208091B2053B
S12318000E94A62080915604909157040E94A62080914B0590914C05969587950E94A6208B
S123182089B1881F8827881F90E0909361048093600489B190E080749070909363048093C3
S1231840620489B190E080729070909365048093640489B190E0807190709093670480933F
S1231860660486B190E0827090709093690480936804E0914104F0E0F0936B04E0936A04F9
S1231880E050FF4FE081F0E0F0936D04E0936C04EE0FFF1FE15FFA4F8081918190936F0471
S12318A080936E042091DE0430E0220F331FF901E05AFB4F80819181892F990F990BB3E051
S12318C0220F331FBA95E1F7822B0E94A620E091DE04F0E0EE0FFF1FE05AFB4F8081918170
S12318E00E94A6208DEA0E94A6208091DE048F5F8093DE04883010F01092DE040895CF928D
S1231900DF92EF92FF920F931F93CF93DF93A89588E10FB6F89480936000109260000FBEDF
S12319200E94F220882309F48FC50E9483209093DD048093DC048136910509F486C082366F
S1231940910508F041C08D34910509F4E1C18E349105E8F48134910509F49CC082349105DA
S123196068F48932910509F4ABC48433910509F452C58832910509F065C57FC485349105E4
S123198009F4C1C08634910509F05CC545C18335910509F4E7C48435910548F48035910589
S12319A009F42DC38235910509F04CC5A4C38735910509F49BC38835910509F42CC48535D1
S12319C0910509F03FC5DFC38936910509F4C8C28A369105E8F48436910509F435C58536BE
S12319E0910548F48236910509F478C38336910509F028C573C38636910509F4EBC086366A
S1231A00910508F4F8C18736910509F01BC5CFC28037910509F4F8C28137910548F48D3669
S1231A20910509F434C18F36910509F00BC50BC48937910509F467C48A37910509F46BC228
S1231A408837910509F0FEC466C281E60E94A62080EA0E94A6201092DD041092DC040EC0D6
S1231A60E158FA4F80810E94A6208091DC049091DD0401969093DD048093DC04E091DC04A5
S1231A80F091DD04E03AF10558F382E30E94F71F8EE9D8C41092DD041092DC04C0E0D0E000
S1231AA00E94F220882341F1C091DC04D091DD04C03AD10589F40E9483209093DD04809375
S1231AC0DC048E3B910519F4C6E1DAEF15C08091DC040E94A620FBCF0E948320C158DA4FC7
S1231AE088838091DC049091DD0401969093DD048093DC04C0E0D0E021964AEFC030D4074B
S1231B0008F0A2C4CDCFC0E0D0E00E94F220882309F459C00E9483208A3B910509F094C411
S1231B2088E10FB6F89480936000109260000FBE1092DD041092DC043EC0885B0E94A62057
S1231B408DEF0E94A6202091DC043091DD048AEF90E0289FE001299FD00D389FD00D11244B
S1231B6007C0DE010E94E321802D0E94A62021962091DC043091DD042F5F3F4F8AEF90E011
S1231B80AC01249FC001259F900D349F900D112421503040C817D90720F3822F885B8095AE
S1231BA00E94A6208091DC049091DD0401969093DD048093DC048091DC049091DD04843091
S1231BC0910508F4BACF21965AEFC030D50708F03BC49BCF86E60E94A62080EA0E94A62013
S1231BE01092DD041092DC040EC0E75CFA4F80810E94A6208091DC049091DD04019690936C
S1231C00DD048093DC04E091DC04F091DD04E03AF10558F389E916C41092DD041092DC048D
S1231C2000E010E00E94F220882349F1C091DC04D091DD04C03AD10591F40E948320909307
S1231C40DD048093DC04893B910519F406E11AEF16C0E091D604F091D704099510C00E94C8
S1231C608320C75CDA4F88838091DC049091DD0401969093DD048093DC0400E010E00F5FA7
S1231C801F4F8AEF0030180708F0DEC3CBCF8DE60E94A62089E00E94A620809140019091B8
S1231CA041010E94A6208091400190914101892F99270E94A62080914601909147010E947E
S1231CC0A6208091460190914701892F99270E94A62080912401909125010E94A6208091A3
S1231CE0240190912501892F99270E94A620809137010E94A620809136010E94A620AAE0A9
S1231D00B0E00E94E321802D0E94A62082E99AC31092DD041092DC04C0E0D0E00E94F220A3
S1231D208A3008F461C00E948320909341018093400100914001109141010E948320982F09
S1231D408827800F911F90934101809340010E948320909347018093460100914601109155
S1231D6047010E948320982F8827800F911F90934701809346010E948320909325018093B7
S1231D80240100912401109125010E948320982F8827800F911F90932501809324010E9480
S1231DA08320809337010E948320809336010E948320AAE0B0E0082E0E94F0210E94941A0A
S1231DC00E948320823B910551F40E949303E091D604F091D7040995CFE6DAEF05C0E091F1
S1231DE0D604F091D704099521964AEFC030D40708F02AC393CF85E60E94A62083E10E9430
S1231E00A6201092DD041092DC040EC0EA5FFD4F80810E94A6208091DC049091DD0401969D
S1231E209093DD048093DC04E091DC04F091DD04EA30F10558F380913D010E94A6208091D1
S1231E403E010E94A62083E00E94F81F80914B010E94A62080914C010E94A62080914D01D1
S1231E600E94A62080914E010E94A620809138019091390166E070E00E947F21CB010E9443
S1231E80A620809148010E94A620AEE6B1E00E94E321802D0E94A6208AE90E94A6208CE689
S1231EA00E94A62084E10E94A6201092DD041092DC040EC0E05BFA4F80810E94A620809118
S1231EC0DC049091DD0401969093DD048093DC04E091DC04F091DD04EA30F10558F31092DE
S1231EE0DD041092DC040EC0E05BFA4F80890E94A6208091DC049091DD0401969093DD042A
S1231F008093DC04E091DC04F091DD04EA30F10558F383E997C20E94940B96C20E94832019
S1231F20C82FD0E00E948320C817D90709F08CC20E9483208C019093DD048093DC040E9440
S1231F4083200817190709F07FC20E9483208639910509F079C28091DC04C158DA4F4DC053
S1231F600E94F2208530D0F6FBCF0E948320C82FD0E00E948320C817D90709F065C20E94B2
S1231F8083208C019093DD048093DC040E9483200817190709F058C20E94832088399105E3
S1231FA009F052C28091DC04C75CDA4F26C00E94F2208530D0F6FBCF0E948320C82FD0E008
S1231FC00E948320C817D90709F03EC20E9483208C019093DD048093DC040E9483200817D3
S1231FE0190709F031C20E9483208F3A910509F02BC28091DC04CA59DE4F888325C20E9472
S1232000F2208530C8F6FBCFC0E0D0E00E94F220823080F10E9483200E9483208F3891055F
S123202009F012C21092DD041092DC041CC0EA59FE4F108180E70E94A62082E00E94A62034
S12320408091DC040E94A620812F0E94A6208FE80E94A6208091DC049091DD04019690937F
S1232060DD048093DC04E091DC04F091DD04E03AF105E8F221965AEFC030D50709F4E4C17D
S1232080C5CF0E9483208C010E948320D82FCC27C00FD11F0E9483208C019093DD048093EF
S12320A0DC040E9483200817190709F0CDC10E948320883A9105A9F4DE010E94EB21E0701A
S12320C08091DC049091DD04E82BF92BF093DD04E093DC04DE010F010E94FC2112BC11BCD2
S12320E0B3C1E091D604F091D70409950E94F220853038F6FBCFCC24DD240E94F22083306A
S1232100C0F10E9483208C010E948320EC010E9483208D3A910509F097C1FC2EEE24E00EE9
S1232120F11ED7010E94E321802D90E0D70111960E94E321002D10E0102F0027080F191FFA
S123214084E50E94A62084E00E94A620802F0E94A6208E2D0E94A620EF2CFF248E2D0E9409
S1232160A620012F1127802F0E94A6208BEA0E94A6200894C11CD11C80E0C8168AEFD8063E
S123218009F462C1BACFCC24DD240E94F2208330C0F10E9483208C010E948320EC010E94E3
S12321A083208A3A910509F04FC1FC2EEE24E00EF11ED7010E94E321802D90E0D7011196C2
S12321C00E94E321002D10E0102F0027080F191F85E50E94A62084E00E94A620802F0E9494
S12321E0A620012F1127802F0E94A6208E2D0E94A620EF2CFF248E2D0E94A6208AEA0E94FC
S1232200A6200894C11CD11C40E0C4164AEFD40609F41AC1BACFC0E0D0E00E94F220882371
S123222059F00E948320873A910509F00DC1E091D604F091D704099521965AEFC030D507DD
S123224009F402C1EACFC0E0D0E00E94F220882369F00E9483208039910509F0F5C00E9415
S12322609300E091D604F091D704099521968AEFC030D80709F4E8C0E8CFC0E0D0E00E9435
S1232280F2208823B1F00E948320873D910509F0DBC080915C0490915D04ADE6B1E0082E5C
S12322A00E94F02112BC11BCE091D604F091D704099521964AEFC030D40709F4C5C0DFCF9C
S12322C0C0E0D0E00E94F2208823B1F00E948320863D910509F0B8C080915C0490915D04A8
S12322E0AEE6B1E0082E0E94F02112BC11BCE091D604F091D704099521965AEFC030D50720
S123230009F4A2C0DFCFC0E0D0E00E94F220823010F10E948320892B09F096C00E94832068
S123232086389105C1F489E70E94A62085E00E94A6208FEC0E94A6208FE30E94A62083E1CA
S12323400E94A6208CE80E94A62080E70E94A62086E80E94A62021968AEFC030D80709F494
S123236073C0D3CFC0E0D0E00E94F220823008F44CC00E948320892B09F047C00E94832088
S12323808C3A910509F060C083E50E94A62088E00E94A6208091BD049091BE040E94A62007
S12323A08091BD049091BE04892F99270E94A62080917C0590917D050E94A62080917C0555
S12323C090917D05892F99270E94A62080917405909175050E94A6208091740590917505C4
S12323E0892F99270E94A6208091C9059091CA050E94A6208091C9059091CA05892F99277B
S12324000E94A6208CEA0E94A62021964AEFC030D407D1F0A9CFC0E0D0E00E94F2208230C8
S123242058F00E948320892B79F40E9483208B3C910511F40E94120121965AEFC030D507C2
S123244019F0EBCF0E94A620A895DF91CF911F910F91FF90EF90DF90CF9008950F931F9323
S1232460CF93DF9310929105109290050E94EF1F259A249A000001E000938F0500934D05FB
S123248000937A05000000934E05209A219A219A209A109236051092B6051092380510929B
S12324A07E050000000010927B0510922B05229A239A3A9A009329051092370542980000DB
S12324C00000529853983B98439A3C983E983F98289829982D982C982A982B980000399892
S12324E0389857985698559854980E94FA1FAAE5B1E00E94E321802D8093C3040E94431A4B
S12325000E94941A0E94DD1F0E943D060E9497040E94A700A1EDB7E00E94E321802D90E076
S1232520813009F491E0909340040093290510923705A7E0B0E00E94E321802D12BC11BC6D
S123254085FF9BC080912401909125019F7D90932501809324010E9493030E94E00312BCF3
S123256011BC12BC11BC0E94930086E0AAE0B0E0082E0E94F02189E1ABE0B0E0082E0E94F4
S1232580F0218EE1ACE0B0E0082E0E94F021AEE0B0E0082E0E94F02120E030E0F901EA5F58
S12325A0FD4F8081D901A25ABE4F082E0E94F0212F5F3F4F2A30310589F780914B01A9E6E6
S12325C0B1E0082E0E94F02180914C01AAE6B1E0082E0E94F02180914D01ABE6B1E0082E5E
S12325E00E94F02180914E01ACE6B1E0082E0E94F02120E030E0F901E05BFA4F8081D9014F
S1232600AE58BE4F082E0E94F0212F5F3F4F2A30310589F720E030E0F901E05BFA4F8089F7
S1232620D901A458BE4F082E0E94F0212F5F3F4F2A30310589F780917305A1E7B1E0082EC6
S12326400E94F021809138019091390166E070E00E947F21ADE0B0E0062E0E94F02184E1DD
S1232660ADE6B1E0082E0E94F02181EEAEE6B1E0082E0E94F02112BC11BC0E947E000E946F
S1232680120112BC11BC0E946100809124019091250185FD06C0000081E080938F058093A5
S12326A04D0580914A01882311F480E801C080E480935C0110924F04809138019091390121
S12326C08D5A9D4030F08CEA9DE090933901809338011092B20486B3866086BB78948AEA3E
S12326E00E94A62080E00E94A62085E50E94A62086B1829581708093C504000081E0809345
S1232700290580914004882311F0529A5A9A80914004882359F08BB18695869580958170E5
S1232720880F880F9BB19B7F982B9BB921E020933705A8958091B5049091B6048E379105BD
S123274030F18091B204882311F580919005909191059F7E90939105809390050000000001
S1232760209329052093B204809190059091910580629093910580939005809190059091A4
S123278091059062909391058093900540C02091B204213009F03BC08091B5049091B604FB
S12327A086359105A0F500000000000080919005909191058F7D9093910580939005809154
S12327C0900590919105877F9093910580939005109236051092B6051092380510927E0504
S12327E010927B0510922B0520938F0520934D0520937A051092B2048091900590919105AE
S12328009F7D90939105809390051092B0042091B2042130A1F48091B004882359F00000DB
S12328200000809190059091910588609093910580939005209329052093370519C01092A3
S1232840B00481E080938F0580934D0580937A051092B0041092B3001092BC041092BB0453
S12328608091640190916501892B11F41092290580914F04833009F4E1C0843018F48823AE
S123288071F074C0853009F428C2853008F439C1863009F4CBC1873009F0DEC25CC280919A
S12328A0B3049091B4048536910508F4D8C2E0914F04F0E080917800909179008C7F65E096
S12328C070E00E947F21EE0FFF1FE057FB4F7183608380914F04C82FD0E0E0914F04F0E050
S12328E0EE0FFF1FE05BFB4F80819181E0914F04F0E0EE0FFF1FE057FB4F20813181880F07
S1232900991F880F991F820F931F880F991F6AE070E00E947F21CC0FDD1FC05BDB4F798326
S123292068831092B4041092B30401E000934F0481E480937C000E947F0C0E940807909339
S12329403B0180933A018091640190916501892B09F480C280916401909165010197909341
S12329606501809364010093290574C28091B3049091B4048536910508F471C290914F04E9
S12329804091CC04842F83708450990F990F980FE92FF0E0EE0FFF1FEA5DFE4F8081918177
S12329A02091780030917900820F931F96958795918380831092B4041092B304A89580910E
S12329C04F04813051F5842F0E94480690935304809352042091CC04E22FF0E0E370F0700E
S12329E0EE0FFF1FEA5DFE4F8081918164E070E00E9493217093E6046093E504222341F4E4
S1232A0080916004909161040E94500B8093B70582E080934F0485E40EC08081918162E097
S1232A2070E00E949321709355046093540483E080934F0484E480937C0011C28091B304EA
S1232A409091B4048536910508F409C2E0914F04F0E0809178009091790096958795969558
S1232A608795EE0FFF1FE057FB4F9183808380914F04C82FD0E0E0914F04F0E0EE0FFF1FC9
S1232A80E05BFB4F80819181E0914F04F0E0EE0FFF1FE057FB4F20813181880F991F880F31
S1232AA0991F820F931F880F991F6AE070E00E947F21CC0FDD1FC05BDB4F79836883109247
S1232AC0B4041092B30484E080934F0480915C0180937C000E947F0CA8958091CC048F5FE1
S1232AE08093CC04843010F01092CC048091CC04982F917090932A05869581708093760534
S1232B00AEC18091B3049091B4048159914008F4A6C180914A018823F9F0E0914F04F0E00F
S1232B208091780090917900EE0FFF1FE057FB4F9183808380914F04C82FD0E0E0914F04EC
S1232B40F0E0EE0FFF1FE057FB4F8081918164E070E00E94932138C0E0914F04F0E080916B
S1232B60780090917900EE0FFF1FE057FB4F9183808380914F04C82FD0E0E0914F04F0E0ED
S1232B80EE0FFF1FE05BFB4F00811181E0914F04F0E0EE0FFF1FE057FB4F808191810E9499
S1232BA03A079C01220F331F280F391FC80143E0880F991F4A95E1F7801B910B820F931FB5
S1232BC06AE070E00E947F21CC0FDD1FC05BDB4F79836883E0914F04F0E0EE0FFF1FE0572C
S1232BE0FB4F8081918164E070E00E9493217093E8046093E7041092B4041092B30485E0A5
S1232C0080934F0487E880937C002091C50486B18295817030E090E02817390709F41AC1BC
S1232C20E091D604F091D704099514C18091B3049091B4048536910508F411C1E0914F04F2
S1232C40F0E080917800909179009695879596958795EE0FFF1FE057FB4F9183808380912B
S1232C604F04C82FD0E0E0914F04F0E0EE0FFF1FE05BFB4F80819181E0914F04F0E0EE0F7E
S1232C80FF1FE057FB4F20813181880F991F880F991F820F931F880F991F6AE070E00E94D2
S1232CA07F21CC0FDD1FC05BDB4F79836883E0914F04F0E0EE0FFF1FE05BFB4F8081918126
S1232CC09093E4048093E3041092B4041092B30487E080934F0483E4B9C08091B3049091A2
S1232CE0B404893C910508F4BAC0E0914F04F0E08091780090917900EE0FFF1FE057FB4FF4
S1232D0091838083A0914F04B0E0E0914F04F0E0EE0FFF1FE05BFB4F20813181E0914F0439
S1232D20F0E0EE0FFF1FE057FB4F80819181820F931F96958795AA0FBB1FA05BBB4F119647
S1232D409C938E931092B4041092B30486E080934F0482E47BC08091B3049091B4048536A3
S1232D60910508F47CC0E0914F04F0E08091780090917900969587959695879590E0EE0FCF
S1232D80FF1FE057FB4F91838083E0914F04F0E0EE0FFF1FE05BFB4F8081918184369105E2
S1232DA00CF5A0914F04B0E0E0914F04F0E0EE0FFF1FE05BFB4F40815181E0914F04F0E09F
S1232DC0EE0FFF1FE057FB4F20813181CA01880F991F840F951F820F931F969587959695EA
S1232DE0879519C0A0914F04B0E0E0914F04F0E0EE0FFF1FE05BFB4F20813181E0914F047B
S1232E00F0E0EE0FFF1FE057FB4F80819181820F931F96958795AA0FBB1FA05BBB4F119666
S1232E209C938E93E0914F04F0E0EE0FFF1FE05BFB4F808191819093E2048093E104109254
S1232E40B4041092B30410924F0486E480937C000E947F0CA89503C081E080934F0480916A
S1232E60B3049091B40401969093B4048093B3048091B5049091B6048B58924008F45BC011
S1232E808091B4058F5F8093B4059091B4058091B505981708F452C01092B40580915E047A
S1232EA090915F04E091D105FF27E7FDF095EE56FA4F208130E08217930754F48091B20533
S1232EC0843634F48091B2059091B305890F17C080915E0490915F04E091D105FF27E7FDB4
S1232EE0F095EE56FA4F208130E0821793074CF08091B20582302CF08091B205815080935A
S1232F00B2058091B205E091D105FF27E7FDF095EE56FA4F2089992787FD909530E028176A
S1232F20390764F4E091D105FF27E7FDF095EE56FA4F808901C081E08093B2058091B504D3
S1232F409091B6048739910508F46DC020915C0430915D048091480190E0499628173907B8
S1232F600CF061C08091320590913305019690933305809332052091320530913305809161
S1232F803405909135052817390708F440C010923305109232052091B5043091B604809175
S1232FA02C0590912D050A972817390730F49091300580913105890F15C02091B504309110
S1232FC0B60480912C0590912D0549968217930758F49091300580912F05891728F48091D8
S1232FE030058150809330059091300580912E05891718F480912E0508C0909130058091C6
S12330002F05981720F480912F05809330058091B5049091B6048A58924038F480912E055F
S12330208093300502C01092300580914E0482FF1BC08091B5049091B604805D9740A0F4FF
S123304020915C0430915D048091480190E00596281739074CF481E08093C7048091900530
S123306090919105916007C01092C70480919005909191059E7F9093910580939005809184
S123308024019091250192FF27C02091B5043091B604809152019091530182179307E0F483
S12330A02091B5043091B60480915401909155012817390788F420915C0430915D0480910B
S12330C0480190E005962817390734F48091900590919105946005C080919005909191057E
S12330E09B7F90939105809390050E946A080E94A607809124019091250180FF6DC08091B4
S1233100510180FF11C080912805883C28F0809130058823B9F41AC09091300580912805E3
S123312086958917A8F012C08091510182FF10C080912805883C60F0809190059091910503
S123314096FF04C081E080937B0502C010927B058091510184FF16C080912805883C28F064
S12331608091B20518165CF12EC02091B20580912805332727FD3095869590E08217930773
S123318024F121C08091510186FF1FC080912805883CD8F02091B5043091B6048091560157
S12331A0909157018217930770F420915E0430915F048091C40490E08217930724F481E0CF
S12331C080932B0502C010922B0580912805883C38F01092280504C010927B0510922B0563
S12331E0809128058F5F8093280591CA1F920F920FB60F9211248F939F938091D2058F5FED
S12332008093D2058091D205882369F1809190059091910590619093910580939005109282
S1233220B20480919005909191059F7D909391058093900500000000000080919005909133
S123324091058F7D90939105809390058091900590919105877F9093910580939005109201
S1233260B6041092B50478949F918F910F900FBE0F901F901895CF93DF9320E030E01EC0B0
S1233280A92FB0E0FD01EE0FFF1FEF01CF5EDA4F88819981892B81F0E651FC4F0190F08197
S12332A0E02D8081AA50BC4F9C91892329F4888199810197998388832F5F3F4F922F809131
S12332C0D9032817E8F2DF91CF9108950F931F9380912404909125049093DB058093DA05BC
S12332E08091240490912504499708F455C08091D205882349F088EE9DEF90932904809325
S123330028041092D2050CC01092B8041092B704809124049091250490932904809328046B
S12333201092B9048091B5049091B604809128049091290490937D0580937C0520917C058F
S123334030917D05009126041091270440E050E060E070E489E191E00E94C821CA01B901D0
S12333602CE330E040E050E00E94602120EC30E0A901049F9001059F300D149F300D1124B7
S12333802050324040E050E00E94A6213093B6042093B5041092D20578941F910F91089533
S12333A01F920F920FB60F9211242F933F934F935F936F937F938F939F93AF93BF93EF9336
S12333C0FF932091DF043091E0048091D7039091D8032817390798F08091840090918500F5
S12333E0909325048093240410928500109284001092E0041092DF040E94661909C08091EF
S1233400DF049091E00401969093E0048093DF040E943B197894FF91EF91BF91AF919F915A
S12334208F917F916F915F914F913F912F910F900FBE0F901F9018951F920F920FB60F92D9
S123344011248F939F9380910E0490910F04019690930F0480930E049F918F910F900FBEDA
S12334600F901F9018951F920F920FB60F9211248F9381E08093290578948F910F900FBE04
S12334800F901F9018951092800081EF9FEF909389008093880085EF9FEF90938B00809303
S12334A08A0080E88093810080EC9AED909385008093840083E090E09093270480932604F2
S12334C0809126049091270480688093810081E080936F0052985398259A249A80938F0509
S12334E080934D0580937A05A2E0B2E00E94E321802D80931204A1E0B2E00E94E321802DDB
S123350080931304809113048E3039F080911304873119F087E18093130480916900826097
S123352080936900E89A0895E1EBF0E010821092B6001092B2001092B300209A219A219A8D
S1233540209A109236051092B6051092380510927E05000086E0808384E680937005089577
S12335608130B9F41092360510927E0580915001843031F41092B6051092380510922B049F
S12335801092E1051092E00510922A041092B1000895823059F41092B6051092380510927B
S12335A0DF051092DE0510922B0415BC08951F920F920FB60F9211242F933F934F935F930A
S12335C06F937F938F939F93AF93BF93EF93FF93F89480912A04843019F481E00E94B01A7E
S12335E07894FF91EF91BF91AF919F918F917F916F915F914F913F912F910F900FBE0F9050
S12336001F9018950F931F9380915004909151040A9714F487E003C08091C70486E08093F3
S1233620B1001092B2008091B5049091B604845F914018F41092C80516C08091B5049091EC
S1233640B6048D56974020F08EE08093C8050BC08091B5049091B60464E670E00E947F2148
S123366065506093C805E091C805F0E0E05FFD4F8081809337018091C704882329F020919B
S1233680490580913C0108C0E091B904F0E0E75CFA4F808120913C01829FC001112490930F
S12336A02505809324058091B5049091B6048059914048F5809124019091250182FF19C03D
S12336C0809124059091250520913D01820F911D909325058093240580919005909191054D
S12336E0846090939105809390058EE1809326053FC080919005909191058B7F90939105B5
S12337008093900535C080919005909191058B7F909391058093900580912605823028F03A
S123372080912605815080932605E0912405F091250580913D0120913D0140912605E80FC4
S1233740F11D8EE190E0841B910930E0AC01429FC001439F900D529F900D11246EE170E0FF
S12337600E947F21E61BF70BF0932505E09324058091C704882309F0A3C18091D10587FD68
S12337803EC08091D1058F30D4F5E091B904F0E0E65CFA4F6081E091B904F0E0E75CFA4FC4
S12337A0408100912405109125058091BA052091D105E0913C0170E0641B710990E04AE0D7
S12337C0240290011124821B930B9C01629FC001639F900D729F900D11246AE070E00E94A1
S12337E09321F0E06E9FC0016F9F900D7E9F900D1124800F911F9093250580932405809100
S1233800BC0587FD3EC08091BC058930D4F5E091B904F0E0E75BFA4F6081E091B904F0E0A5
S1233820E75CFA4F408100912405109125058091CC052091BC05E0913C0170E0641B710967
S123384090E04AE0240290011124821B930BAC01649FC001659F900D749F900D11246AE062
S123386070E00E949321F0E06E9FC0016F9F900D7E9F900D1124800F911F909325058093C7
S12338802405809124019091250184FF5CC020917C0430917D0480915C0490915D0428173A
S12338A03907FCF480915C0490915D0420917C0430917D04821B930B64E070E00E94932149
S12338C08091BA04861710F46093BA048091BA048A3018F089E08093BA048091490180938A
S12338E02705309127053430C8F08091240590912505E091BA04F0E0EA5FFD4F2081820F44
S1233900911D90932505809324053150309327058091900590919105806109C01092BA0495
S12339201092270580919005909191058F7E909391058093900580915C0490915D049093D4
S12339407D0480937C04809124019091250191FFB4C08091C504882309F0AFC08091720559
S12339608F5F809372059091720580917305981708F4A6C010927205809158049091590495
S1233980E091BC05FF27E7FDF095E05BFA4F208130E028173907B4F480915804909159041B
S12339A0E091BC05FF27E7FDF095E05BFA4F2081821B910962E070E00E9493216C59609346
S12339C070052BC08091580490915904E091BC05FF27E7FDF095E05BFA4F208130E0821709
S12339E09307DCF4809170051816BCF4E091BC05FF27E7FDF095E05BFA4F808120915804A2
S1233A003091590490E0821B930B62E070E00E94932184E6861B8093700580919005909197
S1233A2091059D7F909391058093900520917005E091BC05FF27E7FDF095E05BFA4F8089FB
S1233A40332727FD309590E08C599F4F8217930754F4E091BC05FF27E7FDF095E05BFA4F1C
S1233A6080898C591EC020917005E091BC05FF27E7FDF095E05BFA4F4089332727FD3095FF
S1233A8084E690E0841B910928173907CCF4E091BC05FF27E7FDF095E05BFA4F908984E608
S1233AA0891B8093700580919005909191059260909391058093900503C084E68093700571
S1233AC020912405309125058091B70590E0829FB001839F700D929F700D1124882777FD69
S1233AE08095982F24E630E040E050E00E94A6213093250520932405209166043091670403
S1233B0080913F0190E0C296281739070CF046C0809124019091250181FF40C0809166048F
S1233B2090916704C397D4F040913E0180913E01209166043091670460913F0190E070E03F
S1233B406E5C7F4FFC01E29FC001E39F900DF29F900D11240E947F21461B03C080913E0152
S1233B60482F50E08091240590912505480F591F5093250540932405809144019091450180
S1233B80909343018093420180919005909191058260909391058093900511C0809190054D
S1233BA0909191058D7F90939105809390058091400190914101909343018093420180915A
S1233BC04A01882371F020912405309125058091700524563040992787FD9095280F391F5D
S1233BE00DC02091240530912505809170052C593F4F992787FD9095281B390B30932505B9
S1233C00209324058091490590914A0583FF1CC0E0912405F091250520915E018091240508
S1233C209091250564E170E00E94932130E0629FC001639F900D729F900D11248E0F9F1F9B
S1233C409093250580932405809124019091250190FF4CC080915004909151048238910594
S1233C600CF044C0809124059091250520914B01820F911D9093250580932405E091500431
S1233C80F091510460913C0120914B0182E890E08E1B9F0B70E0AB01849FB001859F700D81
S1233CA0949F700D11248FEF90E0FB01E89FB001E99F700DF89F700D1124882777FD809573
S1233CC0982F30E040E050E00E94602120E43FE140E050E00E94A621809124059091250534
S1233CE0820F931F9093250580932405209124053091250580913C0145EF849FC001112494
S1233D008217930754F480913C01849FC001112490932505809324050BC08091240590910E
S1233D2025051816190624F0109225051092240580912405909125059093BC048093BB0423
S1233D40809190059091910592FF08C0109236051092B6051092380510927E0578941F91AF
S1233D600F9108951F920F920FB60F9211242F933F934F935F936F937F938F939F93AF9303
S1233D80BF93EF93FF93F89420912A04223039F0243009F44FC0213009F051C01CC080912B
S1233DA0E0059091E1058F3F9105D1F1C8F18091E0059091E1058F5F8093B3008091E0058D
S1233DC09091E1058F5F90409093E1058093E00520932A0434C00E94021B8091BB04909194
S1233DE0BC049093E1058093E0058091E0059091E1058F3F9105A1F098F08091E00590916D
S1233E00E1058F5F8093B3008091E0059091E1058F5F90409093E1058093E00582E007C01F
S1233E208091E0059091E1058093B30084E080932A0405C081E00E94B01A10922A047894A8
S1233E40FF91EF91BF91AF919F918F917F916F915F914F913F912F910F900FBE0F901F9044
S1233E6018951F920F920FB60F9211242F933F934F935F936F937F938F939F93AF93BF9340
S1233E80EF93FF93F89420912B04223039F0243009F453C0213009F053C020C08091DE058E
S1233EA09091DF058F3F910591F088F08091DE059091DF058F5F87BD8091DE059091DF0578
S1233EC08F5F90409093DF058093DE0533C08091DE059091DF0587BD84E024C08091BB04DB
S1233EE09091BC049093DF058093DE0524E025BD16BC8091DE059091DF058F3F9105A9F032
S1233F00A0F08091DE059091DF058F5F87BD8091DE059091DF058F5F90409093DF05809311
S1233F20DE0582E080932B040BC08091DE059091DF0587BD20932B0403C082E00E94B01A7B
S1233F407894FF91EF91BF91AF919F918F917F916F915F914F913F912F910F900FBE0F90E6
S1233F601F9018951F920F920FB60F9211242F933F934F935F936F937F938F939F93AF93E2
S1233F80BF93EF93FF93F89480912B04843019F482E00E94B01A7894FF91EF91BF91AF91B0
S1233FA09F918F917F916F915F914F913F912F910F900FBE0F901F90189500000000109234
S1233FC07B0510922B0515BCEEE6F0E080818360808384E085BD16BC82E187BD089511B8AA
S1233FE08FEF84B915B887B98AB90895089508950895089588E98093C10083E18093C40021
S123400089E296E09093E7058093E6059093E3058093E20589EE95E09093E5058093E405B4
S123402090936A06809369061092E8051092790508951F920F920FB60F9211248F939F93DA
S1234040EF93FF938091E805882311F1E091E605F091E70581918093C600F093E705E09307
S1234060E605E956F64030F089E296E09093E7058093E6058091E80581508093E8058091EE
S1234080E805882329F48091C1008F7D8093C100FF91EF919F918F910F900FBE0F901F909B
S12340A018951F920F920FB60F9211242F938F939F93EF93FF938091C600E0916906F09100
S12340C06A068083809179058F5F809379058091690690916A06019690936A06809369069E
S12340E08952964030F089EE95E090936A0680936906FF91EF919F918F912F910F900FBE5E
S12341000F901F90189580917905882319F48FEF9FEF0895F8948091790581508093790533
S1234120E091E405F091E5052191F093E505E093E405E952F64030F089EE95E09093E505B1
S12341408093E4057894822F90E00895982F8091E8058F33E0F78091E805803418F080E01D
S123416090E00895F8948091E8058F5F8093E805E091E205F091E30590838091E2059091C9
S1234180E30501969093E3058093E2058956964030F089E296E09093E3058093E2058091CB
S12341A0C10080628093C100789481E090E00895CF93DF93EC0104C00E94A62081112196D4
S12341C088818823C9F781E090E0DF91CF9108958CE294E00E94D820089584E394E00E9493
S12341E0D82008958091790590E00895CF92DF92EF92FF920F931F93CF93DF93CDB7DEB765
S123420029970FB6F894DEBF0FBECDBF8C01F62EE42EDE011196E7E3F4E089E001900D9213
S12342208150E1F749E06E010894C11CD11CFF2081F089E090E0841B91092F2D30E082172C
S1234240930738F04150F601E40FF11D8CE28083FF244150F601E40FF11DC8016AE070E08F
S12342600E947F21805D8083C8016AE070E00E947F218B01672B11F4FF2019F085E08F151F
S1234280B0F619E01E197E010894E11CF11C07C0F701E10FF11D80810E94A6201F5F193032
S12342A0B8F329960FB6F894DEBF0FBECDBFDF91CF911F910F91FF90EF90DF90CF900895B0
S12342C0629FD001739FF001829FE00DF11D649FE00DF11D929FF00D839FF00D749FF00D8E
S12342E0659FF00D9927729FB00DE11DF91F639FB00DE11DF91FBD01CF0111240895AA1B1B
S1234300BB1B51E107C0AA1FBB1FA617B70710F0A61BB70B881F991F5A95A9F78095909501
S1234320BC01CD01089597FB092E07260AD077FD04D0E5DF06D000201AF4709561957F4FA8
S12343400895F6F7909581959F4F0895A1E21A2EAA1BBB1BFD010DC0AA1FBB1FEE1FFF1F0A
S1234360A217B307E407F50720F0A21BB30BE40BF50B661F771F881F991F1A9469F76095E8
S12343807095809590959B01AC01BD01CF01089597FB092E05260ED057FD04D0D7DF0AD0DC
S12343A0001C38F450954095309521953F4F4F4F5F4F0895F6F790958095709561957F4F15
S12343C08F4F9F4F0895F999FECFB2BDA1BDF89A119600B40895F7DFE02DF5DFF02D089549
S12343E0F999FECFB2BDA1BD00BC11960FB6F894FA9AF99A0FBE0895F3DF012CF1DF112444
S12344000895FFCF01020304050601020304050601020304050601020304050601020304CF
S123442005060102030405062F00010002000300040005000600070008003228E80390012F
S123444006141E3C581B581B88136419121E01010203040A0411C4098813C4096400DCE631
S12344604003020A1432469650000000000000000000000000000000000000000000000077
S1234480000000000000000000000000000000000000000000000000000000000000000018
S12344A0000000000000000000000102030405060708090A0B0C0D0E0F100102030405065B
S12344C00708090A0B0C0D0E0F100102030405060708090A0B0C0D0E0F1014161718191A51
S12344E01B1C1D1E1F2021222324191A1B1C1D1E1F2021222324252627271E1F20222324B0
S123450025262728292A2B2C2D2E000204060708090A0C0E28262422201E1E1E1E1E1E1E2A
S12345201E1E1E1EF0FF80BBE0880465484BA438022BF0207019CC13860F440CC209D00769
S12345404C061B052A046A03D1025602F201A1015F012801FB00D600B7009D0087007500E0
S1234560660059004D0044003C0034002E0029002500F0FF80BBE0880465484BA438022B64
S1234580F0207019CC13860F440CC209D0074C061B052A046A03D1025602F201A1015F01EB
S12345A02801FB00D600B7009D0087007500660059004D0044003C0034002E002900250071
S12345C0F0FF80BBE0880465484BA438022BF0207019CC13860F440CC209D0074C061B05CF
S12345E02A046A03D1025602F201A1015F012801FB00D600B7009D008700750066005900F3
S12346004D0044003C0034002E0029002500F0FF80BBE0880465484BA438022BF0207019E9
S1234620CC13860F440CC209D0074C061B052A046A03D1025602F201A1015F012801FB00BF
S1234640D600B7009D0087007500660059004D0044003C0034002E00290025000000F504FB
S12346607E05AE066C08C00AB30D630F8B10D7118813000000000A000F001E003C00780086
S1234680FA007201E00180028002000008000A000C000E00C80A4A067E048403AC0D641A36
S12346A0002000270032003E0066008E00B202EB02240337034B03560361037003E800D60D
S12346C000C200B0009D008A00780078006500520040002D00190007000000B40006B80B8C
S12346E0B80BB80BB80BB80BB80BB80BB80B2600260029002900290029000201804020107E
S12347002500250025002500250025000102201004080100010001175A5A5A5050505050C0
S123472050505050505050506400030000FA04041B5B481B5B324A000D0A00202020202025
S107474020202020F1
S503023BBF
